:020000040000FA
:1000000083160F3086001D30850083121A308C0055
:10001000840000308E0091000E1017200E181D2055
:100020000E1827200E104E200E1854200C28051EE6
:100030000800051A19280E14080006080F398D004B
:1000400085191116851D111211088D0408000C0860
:1000500046200E104B200E1833280C0884000D0883
:1000600080008C0A08000C088F008C0A1A300F02DE
:100070008F03031941280F0884000008840A8000B8
:1000800036281A3084000D08800008004F300C021A
:1000900003190C28080005190E140800051C080097
:1000A000051850280E1408001A3084008F008F0A9B
:1000B0000008000EF0398600001A8514001E851015
:1000C0000F080C0203196B280F0884000008840332
:0A00D00080008F0A60288C030800EE
:02400E00F13F80
:00000001FF
